:020000040000FA
:1000000001288501860190019101920193019401DB
:10001000AC01AD01AA01AB018316013085000030AF
:100020008600831680308100831200308B0091207F
:100030002921C330810000000B1D1B28C330810023
:100040000B11B521900A1008023A031D2F289001C8
:10005000910A1108C83A031D2F2891016D20051837
:1000600032281B2805183228C330810090019101E5
:1000700000000B1D3828C33081000B11B521900AF8
:100080001008643A031D4D289001910A1108C83ADE
:10009000031D4D2891016D201928A20A031D59281E
:1000A000A10A031D5928A00A031D5928A201A10174
:1000B000A001AA1C6A2805183828AA01AB0A2B0837
:1000C000323A031D3828AB0193214821A201A10136
:1000D000A00119280518AA1438288B30C020030164
:1000E0008620D32003018620D32003018620D3203D
:1000F00003018620D3200800960195000A301502DE
:10010000031C85289500960A7E2800348207303427
:10011000313432343334343435343634373438349B
:100120003934AD208610861106110F308605303027
:10013000860486148610B02086148610B02086149B
:100140008610B0202830C0200C30C0200130C020E4
:100150000800AD20AD20AD20AD20B020B020B020F3
:1001600005308C00F9308D0000008D0BB4288C0B0D
:10017000B228080019308D0000008D0BBC28080043
:100180008E00E6200F3086050E08F0398604061131
:100190008611861486100F3086050E0EF0398604FF
:1001A0008614861008008E00E6200F3086050E08A3
:1001B000F039860406118615861486100F308605E0
:1001C0000E0EF03986048614861008008316F0306F
:1001D000060486008312861106158614060886100A
:1001E000F0398F008614060E86100F398F048F1B8E
:1001F000E628061183160F300605860083120800D4
:10020000031018309E009A019B019C019D01990DDD
:10021000980D970D9A0D9B0D9C0D9D0D9E0B112910
:1002200000341D3084001E211C3084001E211B3030
:1002300084001E211A3084001E2107290330000784
:100240009F009F198000303000079F009F1B800097
:1002500000348130C020EE30D320E130D3202F3065
:10026000D320EC30D320E830D320ED30D320C13080
:10027000C020D230D320E030D320E930D320EC307E
:10028000D320E530D320F030D3202030D320080015
:10029000CA30C02014087C2016088620D3201508F8
:1002A0008620D3203A30D32013087C2016088620DD
:1002B000D32015088620D32008001830A600170880
:1002C000A7001808A8001908A9009701980199012A
:1002D000A301A401A5010310A90DA80DA70DA50D4B
:1002E000A40DA30D20082302031D7C29210824024C
:1002F000031D7C2922082502031C8D292208A50242
:10030000031CA4032408FF3A0319A3032108A40231
:10031000031CA3032008A3020314990D980D970D45
:10032000A60B6B290800B73097001B3098000030EF
:1003300099005D2100218B30C0201B0E0F39031D59
:10034000A4292030D320A8291B0E0F398620D320C2
:100350001B080F398620D3201A0E0F398620D32090
:100360001A080F398620D3200034AC0A2C08283A0A
:10037000031D0800AC01AD0A2D08C83A031D080092
:10038000AD01920A12083C3A031D08009201930A3B
:1003900013083C3A031D08009301940A1408183A04
:0803A000031D08009401080090
:02400E00F13F80
:00000001FF
